:1000000025000000000000000000000000000000CB
:1000100000000000000000000000000000000000E0
:1000200000000000000000000000000000000000D0
:1000300000000000000000000000000000000000C0
:1000400000000000000000000000000000000000B0
:0602E0000000A305240A42
:10040000240A00000000000072000C02E201630AEE
:10041000760A810A8C0A970A8C0A970A8C0A970A2C
:100420008C0A970A8C0A970A8C0A970A8C0A970AF0
:100430008C0AA50AB30ABE0AC90AD40ADF0AEA0A64
:10044000FA0A050B140B1F0BDF0C0600000C26002C
:10045000070C2400110C2B00DF0C38007600030C75
:1004600037006C006A006D006E006F007000710054
:10047000C30C020001098607480AF207B20207040A
:100480000304FB0CD20103070705000000003B0A30
:10049000010986063A0AF207B20207040304FB0CBC
:1004A000D2010307070500000000490A110C2B00C8
:1004B0006C006A006D006E006F00700071007200C9
:1004C000F00C670100080000000000000707710A37
:1004D000EB026E0A110C2B00AC02000800000000B9
:1004E0000008110C2B00000000000008F602790A39
:1004F000240A00000000000000000706800AAC0289
:1005000000080000000000000000000000000000E3
:100510000706560AAC020008AC02030407060305EE
:10052000710300000000000000000000000800004F
:10053000000000000000AC020707A20A1107560ADB
:10054000000000081106560A0008AA020A02EC017F
:10055000000000000707B00A1107560A0000000853
:100560001106560A00080706560AAC02AA02000045
:100570000000000000000000000000080706560A06
:1005800011022D00030C2C000000000000000000F0
:1005900000080706560AAC02AA020000000000008C
:1005A00000000000000000080706560A11022E0095
:1005B000030C2C0000000000000000000008AC024A
:1005C000AA0200000000000000000000000000007F
:1005D0000000000811022F000706F50A030C2C008A
:1005E000000000000000000000086C006A007000BD
:1005F0007100230BAC02AA02000000000000000002
:100600000000000000000000000811023000070692
:10061000100B030C2C00000000000000000000087C
:100620006C006A007100230B0707560AAC02AA028D
:1006300000000000000000000000000000080707A4
:10064000560A6C006A000D028E018F019001910123
:100650004307690B760043040D024306410BC30CAC
:100660008D014306340B690BE90C8E014307690BBE
:100670000F02E00E800F4307690B0F022E004C0B98
:10068000690B0E02E00E000F4306610B0E02E00E36
:10069000800F43064C0B690B0E0718050E06180455
:1006A0002E0738052E0638044E0758054E06580406
:1006B00078077805780678041802060040002600BE
:1006C000690B2704C7040D024306670B310AC705EF
:1006D000690B73006D006E006F00700071006A009E
:0206E0003A0AD4
:021FFE00EA0FE8
:00000001FF
